:020000040000FA
:02000000B12C21
:08000800F000030E8301F1007A
:1000100023308100A20A043022020318A201211415
:10002000A30F1528A40F1528A1144A08003E031990
:100030002E283B1C2C2805162E22013038220000C9
:100040001E30A5000512073038220516063038226A
:10005000A50B2228051242282E222F2823223A30CF
:10006000A6000830F40022080319492001302202BA
:1000700003195520023022020319612003302202A5
:1000800003196D2085010B11710E8300F00E700EA7
:1000900009007920A60B4928C5207920CB2079209A
:1000A000D92079202722792008008C20A60B5528FA
:1000B000C5208C20CB208C20D9208C2027228C207E
:1000C00008009F20A60B6128C5209F20CB209F20E1
:1000D000D9209F2027229F200800B220A60B6D2840
:1000E000C520B220CB20B220D920B2202722B220B6
:1000F000080001082902031CF41401082B02031C48
:10010000741501082D02031CF4168316740885006B
:10011000831201308500080001083002031C7414AA
:1001200001082C02031C741501082E02031CF4168E
:1001300083167408850083120230850008000108C8
:100140003102031C741401082702031CF414010873
:100150002F02031CF41683167408850083120430E2
:100160008500080001083202031C741401082802EB
:10017000031CF41401082A02031C74158316740866
:10018000850083122030850008000310330DBC0069
:10019000D220BF0008000310330D013EBC00D22066
:1001A000C000080000308A003C08DD3E03188A0ABF
:1001B00082003F088A004008820001341D34013467
:1001C00028340134303401343834013440340134BB
:1001D00048340134503401345C3401346034013427
:1001E0006C340134703401347C3401348034013493
:1001F0008C340134903401349C340134A034013403
:10020000AC340134B0340134BC340134C034013472
:10021000CC340134D0340134DC340134E0340134E2
:10022000EC340134F0340134FC3402340034023450
:100230000C340234103402341C34BA013030BE00A5
:10024000351825290630B3001E2A0130B3001E2AB6
:1002500035182D290030B3001E2A0230B3001E2AA3
:10026000351835290030B3001E2A0330B3001E2A8A
:1002700035183D290430B3001E2A0330B3001E2A6E
:10028000351845290030B3001E2A0530B3001E2A58
:1002900035184D290730B3001E2A0030B3001E2A3E
:1002A00035185A2900303E0703195829BE0B1E2A5B
:1002B0003A141E2AB3011E2A3508B900B30A1E2AB1
:1002C00039083506031D6629B3011E2A3518381072
:1002D000351C3814B30A1E2A3508B900B30A1E2A81
:1002E00039083506031D7629B3011E2A3518371241
:1002F000351C3716B30A1E2A3508B900B30A1E2A60
:1003000039083506031D8629B3011E2A3518B71191
:10031000351CB715B30A1E2A3508B900B30A1E2AC0
:1003200039083506031D9629B3011E2A35183711E1
:10033000351C3715B30A1E2A3508B900B30A1E2A20
:1003400039083506031DA629B3011E2A3518B71032
:10035000351CB714B30A1E2A3508B900B30A1E2A81
:1003600039083506031DB629B3011E2A3518371082
:10037000351C3714B30A1E2A3508B900B30A1E2AE1
:1003800039083506031DC629B3011E2A3518B612D1
:10039000351CB616B30A1E2A3508B900B30A1E2A40
:1003A00039083506031DD629B3011E2A3518361221
:1003B000351C3616B30A1E2A3508B900B30A1E2AA0
:1003C00039083506031DE629B3011E2A3518B61172
:1003D000351CB615B30A1E2A3508B900B30A1E2A01
:1003E00039083506031DF629B3011E2A35183611C2
:1003F000351C3615B30A1E2A3508B900B30A1E2A61
:1004000039083506031D062AB3011E2A3518B61011
:10041000351CB614B30A1E2A3508B900B30A1E2AC1
:1004200039083506031D162AB3011E2A3518361061
:10043000351C3614B30A1E2AB3013D1408003A10C5
:10044000851E3A1408003510851935140800340843
:100450003302031C2D2A3308B40008003B10CA03E2
:100460000310C90CC80CC70CC60C03183B140800B9
:10047000C100C10B392A0800C701C801C901A03059
:10048000C600C409441C47144418C714421E47152B
:10049000421AC715C21D4716C219C716421D471773
:1004A0004219C717C21C4814C218C814421C481568
:1004B0004218C815C31E4816C31AC816431E48174B
:1004C000431AC817C31D4914C319C914431D49153C
:1004D0004319C915C31C4916C318C916431C49172B
:1004E0004318C9172130CA000800CB000000CB0B0D
:1004F000762A0800D40A54080F3C0319D401540882
:10050000C5000800D4035408013E031D8A2A0E309A
:10051000D400C50008003608D400C500F13E031C15
:10052000952A0E30D40254088E2A0800CC002110DF
:10053000211C982ACC0B972A0800540AD600D70110
:1005400080305B18D700FF30F723D601D701D801E0
:100550000130F72308005408031DB92A0301F122D2
:10056000CF00DB01CF1B5B144F08031DCD2A7A227D
:10057000AB2A0430CD00E130CE000310540DF5005D
:100580008B13DA248B17D0000314540DF5008B1352
:10059000DA248B17CE005008CD0008005408031D44
:1005A000D42A7508F122DE2A0A08D10075088B13B7
:1005B000DA248B17D20051088A005208F50A080085
:1005C00083169C18E12A8B131C1575089B0076086E
:1005D0009A0055309D00AA309D009C148B17831201
:1005E000080083169C18F22A1C119B009C131C14F3
:1005F0001A08831208000301F122D300D31F032B32
:10060000D313DB01052BD3175B14F5015308F60058
:10061000E0229D229D220800AB22F501CE22D500CA
:10062000D513CE22DA00DA0ACE22DC003D1C342BB0
:1006300007303702031D1F2B8B22BD010C2BB7087F
:10064000031D342B2030360203197A222130360262
:1006500003198222003036020319D4010C3036020D
:100660000319FB22BD010C2B3A1C402B9D229D221D
:100670003A1C402B7A229D229D223A183A2B0C2BB1
:1006800001305502031963230230550203196D230B
:100690000330550203199C23043055020319AB2380
:1006A0004A08003E031D602BA11C602BA1105B1C9F
:1006B0005B2B7A220C2B0730C2004508C3003C227A
:1006C000DC0B162B0C2BCE22D600CE22D700CE224E
:1006D000D8005A08D9001F240800DD0A5D08031D50
:1006E000762B2330DD00DE095E08DF0A5D085E1828
:1006F0005D09E00003305F020318DF0100305F0294
:10070000031D872B6008A700AA00AD00B0000130D0
:100710005F02031D902B6008A800AB00AE00B10083
:1007200002305F02031D992B6008A900AC00AF00E6
:10073000B2005A0896220800CE22D600CE22D70058
:100740000F305705E100E10AE10DE10D5A08F723EA
:10075000E10BA62B0800DD0A5D08031DB52B233035
:10076000DD00DE095E085E1CDF0A5D085E185D09BB
:10077000A700A800A900AA00AB00AC00AD00AE0025
:10078000AF00B000B100B2005F18A701DF18A801E8
:100790005F19A9015F18AA01DF18AB015F19AC014D
:1007A0005F18AD01DF18AE015F19AF015F18B0012E
:1007B000DF18B1015F19B201DF19A701DF19A80124
:1007C000DF19A9015F1AAA015F1AAB015F1AAC0118
:1007D000DF1AAD01DF1AAE01DF1AAF015F1BB001F6
:1007E0005F1BB1015F1BB201203096220800D900C7
:1007F000A701D61BA709A801D619A809A901D71BCB
:10080000A909AA01561BAA09AB015619AB09AC01EB
:10081000571BAC09AD01D61AAD09AE01D618AE0909
:10082000AF01D71AAF09B001561AB009B101561875
:10083000B109B201571AB20959089622080059089D
:10084000A7014030561BA707A030D61BA707A80159
:100850004030571BA807A030D71BA807A90140307C
:10086000581BA907A030D81BA907AA014030561A67
:10087000AA07A030D61AAA07AB014030571AAB0717
:10088000A030D71AAB07AC014030581AAC07A030E3
:10089000D81AAC07AD0140305619AD07A030D619B3
:1008A000AD07AE0140305719AE07A030D719AE07DB
:1008B000AF0140305819AF07A030D819AF07B001C9
:1008C00040305618B007A030D618B007B1014030FC
:1008D0005718B107A030D718B107B20140305818E7
:1008E000B207A030D818B2075908962259089622A4
:1008F00059089622080002303302031C0301D60077
:100900000030D7000130F7233A1C952CB401B30115
:100910004A08003E031D952CD601D701D709FF30A8
:10092000F723C2010C30C3003C223D1C7B2CBD01CF
:10093000F030D600D7017F30F723D601D7013F3002
:10094000F723F030D600D7017F30F7233608D600E2
:100950003708D700FF30F723FF30F723B401B30186
:100960007B2CBA0185018101D401CA01B801B7010C
:10097000B601B901B301B401BD01A201DD01DE017F
:10098000DF010730990083168230810070308F04B8
:100990009F0183128B168B17FF30D600D700D8002B
:1009A000FF30F723D601D701D801FF30F7233A1CD7
:1009B0000C2B7B2C4D088A0075084E0703188A0AF9
:1009C00082000434FF340434FF3405342234053407
:1009D00043340534C4340534F7340634163406344D
:1009E00025340634383406343F340634A234073410
:1009F0002F3407345F340734CE340734D134033412
:100A000007341034C034003400340034C0340034AF
:100A1000003401340034C034003400340034C034B5
:100A200000340F34303400340034003430340034B7
:100A300000340134003430340034003400343034B5
:100A400000340F34033420340F3480340034403405
:100A500000342034003410340034003407340834B7
:100A600000340434003402340034013400340034DF
:100A700007340034803400344034003420340034EF
:100A8000103400340F34013480342A3400340034FC
:100A90000034553455345534AA34AA34AA34FF34BA
:100AA000FF34FF34AA34AA34AA34553455345534AB
:100AB000003400340034553400340034AA34003497
:100AC0000034FF3400340034AA3400340034553488
:100AD0000034003400340034003400345534003421
:100AE0000034AA3400340034FF3400340034AA3413
:100AF0000034003455340034003400340034003401
:100B00000034553400340034AA3400340034FF3447
:100B100000340034AA340034003455340034003436
:100B20000034553455340034AA34AA340034FF3428
:100B3000FF340034AA34AA34003455345534003418
:100B40000034003400340034553455340034AA34B1
:100B5000AA340034FF34FF340034AA34AA340034F9
:100B60005534553400340034003455340034553491
:100B7000AA340034AA34FF340034FF34AA340034D9
:100B8000AA345534003455340334303418348034A6
:100B90000034403400342034003410340034113434
:100BA00000342234003444340034883400340834AF
:100BB000003404340034023400340134003401348D
:100BC0001034023420340434403408348034003487
:100BD0008034003440340034203400341034103475
:100BE0001034203420344034403480348034033492
:100BF00030340E34003480340834403484342034AB
:100C000042341034213400341034003400340034C1
:100C1000103400342134003442341034843420340D
:100C20000834403400348034003400340334303429
:100C30000634803424344034423420348134103437
:100C400042342034243440341834033422340834F9
:100C50008034103440342034203440341034803414
:100C60001034803420344034403420348034103404
:100C7000033422340234A53400345A3400340134AD
:100C800022342034403400340034803400340034C2
:100C9000C034003400348034003400346034003414
:100CA0000034203400340034303400340034243430
:100CB000003400341834003400340C340034003470
:100CC0000834003400340534003400340234003475
:100CD000003403340034003402340034003401346E
:100CE000003400340034C03400340034C0340034E4
:100CF0000034C03400340034303400340034303434
:100D0000003400343034003400340C340034003407
:100D10000C34003400340C34003400340334003418
:100D2000003403340034003403340034003400341D
:100D3000C034003400343034003400340C34003417
:100D400000340334013430342E34C03400340034E1
:100D5000603400340034303400340034183400344B
:100D600000340C34003400340634003400340334CE
:100D7000003400340134803400340034C034003492
:100D8000003460340034003430340034003418341B
:100D9000003400340C3400340034063400340034A1
:100DA0000334003400340134803400340034C0345F
:100DB0000034003460340034003430340034003403
:100DC0001834003400340C34003400340634003459
:100DD0000034033400340034033400340034063467
:100DE000003400340C34003400341834003400343F
:100DF000303400340034603400340034C034003403
:100E000001348034003403340034003406340034B8
:100E100000340C34003400341834003400343034DE
:100E200000340034603400340034C0340034013401
:100E30008034003403340034003406340034003489
:100E40000C340034003418340034003430340034AE
:100E50000034603400340034C034003400340134D1
:100E600030340F34403402340934803401340634D1
:100E7000C03400340334903440340234603480345D
:100E800001343034C03400342434903440341834C5
:100E9000603480340C343034C03409342434903419
:100EA00006341834603403340C34303402340934DA
:100EB0002434013406341834003403340C3401343F
:100EC00030342434C03400340034703400340034FE
:100ED0005C340034003417340034003405340034FA
:100EE00000340134003400340334003400340D3451
:100EF00000340034353400340034D4340034003449
:100F00005034003400344034003400340034C034F1
:100F1000003400347034003400345C340034003465
:100F20001B34003400340534003400340134003400
:100F300000340334003400340D34003400343534CC
:100F400000340034D43400340034503400340034DD
:100F50004034003400340034C03400340034703481
:100F6000003400345C34003400341B34003400346A
:100F700005340034003401340034003403340034C8
:100F800000340D3400340034353400340034D434AB
:100F90000034003450340034003440340234073418
:080FA00000340434073400346E
:02400E00C430BC
:10420000010030001200FF001B000000FE006F00E4
:104210000000F900BF000000E400FF000000900073
:10422000FF0001004000FF0006000000FF001B002F
:104230000000FE006F000000F900BF000000E40075
:10424000FF0001009000FF0006004000FF001B007F
:104250000000FF006F000000FE00BF000000F9003A
:10426000FF000000E400FF0001009000FF000600D6
:0242700040000C
:00000001FF
